:020000040800F2
:10000000D0120020F1080008250700082707000883
:100010002B0700082F070008330700080000000026
:10002000000000000000000000000000370700088A
:1000300039070008000000003B0700083D070008E2
:100040000B0900080B0900080B0900080B09000840
:100050000B0900080B0900080B0900080B09000830
:100060000B0900080B0900080B0900080B09000820
:100070000B0900080B0900080B0900080B09000810
:100080000B0900080B0900080B0900080B09000800
:100090000B0900080B0900080B0900080B090008F0
:1000A0000B0900080B0900080B0900080B090008E0
:1000B0000B0900080B0900080B0900080B090008D0
:1000C0000B0900080B0900080B0900080B090008C0
:1000D0000B0900080B0900080B0900081B2D00087C
:1000E0000B0900080B0900080B0900080B090008A0
:1000F0000B0900080B0900080B0900080B09000890
:100100000B0900080B0900080B0900080B0900087F
:100110000B0900080B0900080B0900080B0900086F
:100120000B0900080B0900080B090008230500084B
:10013000DFF80CD002F016FF004800476501000808
:10014000D0120020EFF30980704780F309887047D0
:10015000EFF30880704780F30888704740BA704713
:10016000C0BA70471CB500241EA103C9CDE9000127
:100170004FF000601D49086000F03CF802F00CFEF2
:1001800002F0C6FE4FF4E13000F0FEF802F02CFB66
:1001900001201749086002F027FB21E002F095FDDD
:1001A000012803D102F020FB012406E002F0BCFC90
:1001B000012801D1022400E0002402F015FB012CEB
:1001C00006D102F011FB02F068FD02F00DFB07E022
:1001D000022C05D102F008FB02F032FD02F004FB14
:1001E000DCE700000301050A035C370008ED00E0CE
:1001F0008481224210B5042000F0DCFB2E48006808
:1002000000EB400080002D49B0FBF1F02C49087054
:100210000846007800EB4001C1EBC0104FF6FF71BB
:1002200001EAC0002749088010BD0146244A12781F
:100230004A434FF0E0235A6100229A611A4612693C
:1002400042F001021A6100BF4FF0E022106910F085
:10025000010F02D010F4803FF6D04FF0E022126977
:1002600022F001024FF0E0231A6100229A617047E8
:100270000146144A12884A434FF0E0235A61002293
:100280009A611A46126942F001021A6100BF4FF0EA
:10029000E022106910F0010F02D010F4803FF6D078
:1002A0004FF0E022126922F001024FF0E0231A61C0
:1002B00000229A617047000004000020001BB70074
:1002C000000000200200002010B590B0044601217B
:1002D000880300F0A3FE0121084600F092FE0C9472
:1002E0000020ADF83400ADF83600ADF83800ADF8B8
:1002F0003C000C20ADF83A000CA9204801F0C3F8EE
:1003000001211E4801F04BF91D4801F07DFA1B4800
:10031000001D01901B48029000200390642004906F
:100320000020059080200690002007900890202053
:10033000099000020A9000200B9001A9104801F0DA
:1003400005FB012240210D4801F05AF901210C481A
:1003500001F027FB10B010BD10B5044600BF4021CE
:10036000064801F0F7F90028F9D04021034801F0D0
:10037000FEF92146014801F07FF910BD0038014027
:10038000580002404400002010B586B00446012108
:10039000682000F043FE0121880400F04CFE744800
:1003A00001F02EF8734801F02FFA0420ADF8140084
:1003B00010208DF8170003208DF8160005A96E484F
:1003C00000F076FB4FF48060ADF8140018208DF833
:1003D000170005A9694800F06BFB4FF40060ADF809
:1003E000140004208DF8170005A9644800F060FB94
:1003F00001940020ADF80800ADF80A00ADF80C003B
:10040000ADF810000C20ADF80E0001A9584801F01D
:100410003AF827208DF8000001208DF80100022015
:100420008DF8020001208DF80300684600F077FA8D
:10043000012240F225514E4801F0BDF801214C48FF
:1004400001F0ADF800204E49086006B010BD30B58F
:100450008DB005460C464748143801F0D5F944489C
:10046000001D029003951020049005940020069032
:10047000802007900020089009900A904FF40050C7
:100480000B9000200C9002A93A48143801F05EFA53
:1004900001228021364801F0B3F8012202213948B7
:1004A00001F08BFA3B208DF8040002208DF8050046
:1004B00001208DF806008DF8070001A800F02FFA42
:1004C0000DB030BD70B505460E4601202C490860C0
:1004D0004FF000040CE000BF4021254801F03AF93C
:1004E0000028F9D0295D224801F0C6F8601C84B2CA
:1004F000B442F0DB00BF40211D4801F02BF9002879
:10050000F9D000201E49086070BD10B503460020D8
:1005100000BF03E00C5C1C54441CE0B29042F9DBC9
:1005200010BD10B5184801F06AFA002111481438BE
:1005300001F037FA4FF49670FFF777FE002010496C
:10054000086010BD70B5044601200D4908602046C2
:1005500002F000FDC5B229462046FFF7B3FF012097
:10056000FFF786FE00200949C1F8880170BD000030
:10057000004800403000024000180140000C0140DB
:100580008801234258040240000002100000234268
:1005900000B585B00020ADF800004FF48270ADF8D2
:1005A00002000020ADF80400ADF80600ADF8080028
:1005B0004FF40070ADF80A000020ADF80C00ADF863
:1005C0000E000720ADF810006946534800F0B8FD52
:1005D0000121514800F059FE05B000BD70B5054637
:1005E0000E46002405E0601CC4B2C82C01DD0020CA
:1005F00070BD0221284600F0CCFE0028F3D0314621
:10060000284600F073FE002405E0601CC4B2C82C2C
:1006100001DD0020ECE70121284600F0BAFE0028A9
:10062000F3D0284600F064FEC0B2E1E770B505469D
:10063000002405E0601CC4B2C82C01DD002070BDA0
:100640000221364800F0A5FE0028F3D029463348A1
:1006500000F04CFE002405E0601CC4B2C82C01DD93
:100660000020ECE701212D4800F093FE0028F3D094
:100670002A4800F03DFEC0B2E1E770B5054600240F
:1006800005E0601CC4B2C82C01DD002070BD022151
:10069000214800F07EFE0028F3D029461E4800F0D5
:1006A00025FE002405E0601CC4B2C82C01DD00203A
:1006B000ECE70121184800F06CFE0028F3D0164842
:1006C00000F016FEC0B2E1E770B50546002405E073
:1006D000601CC4B2C82C01DD002070BD022110488E
:1006E00000F057FE0028F3D029460D4800F0FEFD2B
:1006F000002405E0601CC4B2FF2C01DD0020ECE703
:100700000121074800F045FE0028F3D0044800F01E
:10071000EFFDC0B2E1E70000003C004000300140C6
:1007200000380040704700BFFEE700BFFEE700BF93
:10073000FEE700BFFEE77047704770477047000054
:100740000CB50020019000905E48006840F48030B5
:100750005C49086000BF5B48006800F4003000900E
:100760000198401C0190009818B90198B0F5A06F4D
:10077000F1D15448006810F4003F02D001200090ED
:1007800001E0002000900098012828D14E48006820
:1007900040F010004C4908600846006820F0030053
:1007A0000860084600680860464840684549486057
:1007B0000846406848600846406848600846406807
:1007C00020F0030048600846406840F0010048609F
:1007D00000BF3C48406800F00C000428F9D10CBD73
:1007E00010B5FFF7ADFF10BD10B53648006840F0FA
:1007F00001003449086008464068344908403149DE
:10080000486008460068324908402E49086008469A
:10081000006820F4802008600846406820F4FE004C
:1008200048604FF41F008860FFF7DAFF4FF0006068
:100830002849086010BD10B5002100200022214B7E
:100840005B6803F00C0121B1042906D0082928D1E6
:1008500007E0214B214C236027E0214B1F4C2360F4
:1008600023E0184B5B6803F47010164B5B6803F4CD
:100870008032022303EB904022B91A4B4343174CBA
:1008800023600DE00F4B5B6813F4003F04D0164B60
:100890004343124C236003E0114B43430F4C23604E
:1008A00003E00D4B0D4C236000BF00BF054B5B68A0
:1008B000C3F303130D4CE15C084B1B68CB40074CA2
:1008C000236010BD00100240002002400000FFF82D
:1008D000FFFFF6FE08ED00E000127A0004000020A1
:1008E000001BB70000093D00808D5B000800002060
:1008F0000648804706480047FEE7FEE7FEE7FEE7BA
:10090000FEE7FEE7FEE7FEE7FEE7FEE7E907000891
:100910003101000831490143314A1160704770B517
:10092000002100230F22C4780CB32D4C246804F45A
:10093000E064C4F5E064210AC1F10403CA404478CC
:1009400004FA03F18478144021430901254C067808
:10095000A155047804F01F050124AC4005786D1101
:100960004FF0E02606EB8505C5F8004109E0047864
:1009700004F01F050124AC401B4D0678761145F8A4
:10098000264070BD194A0A400243154B1B1F1A60CE
:10099000704739B1124A121D12680243104B1B1DD9
:1009A0001A6006E00E4A121D126882430C4B1B1D92
:1009B0001A607047042808D14FF0E021096941F01E
:1009C00004014FF0E022116107E04FF0E0210969D6
:1009D00021F004014FF0E022116170470000FA0598
:1009E0000CED00E000E400E080E100E080FFFF1F8C
:1009F00010B50446CA48844208D10121042000F001
:100A000027FB0021042000F023FB46E0C548844278
:100A100008D10121082000F01BFB0021082000F074
:100A200017FB3AE0C048844208D10121102000F0B1
:100A30000FFB0021102000F00BFB2EE0BB4884428E
:100A400008D10121202000F003FB0021202000F02C
:100A5000FFFA22E0B648844208D10121402000F08C
:100A6000F7FA0021402000F0F3FA16E0B148844282
:100A700008D10121802000F0EBFA0021802000F055
:100A8000E7FA0AE0AC48844207D10121801500F062
:100A9000DFFA0021A01500F0DBFA10BD10B501212E
:100AA000084600F0D5FA0021012000F0D1FA10BD6F
:100AB0002DE9F041024600250026002000230024F5
:100AC000002791F803C00CF00F0591F803C01CF04B
:100AD000100F03D091F802C04CEA050591F800C050
:100AE000BCF1000F31D0146800202BE04FF0010C56
:100AF0000CFA00F3B1F800C00CEA03069E4220D1C4
:100B000083004FF00F0C0CFA03F7BC4305FA03FC0B
:100B10004CEA040491F803C0BCF1280F06D14FF051
:100B2000010C0CFA00FCC2F814C00AE091F803C0F2
:100B3000BCF1480F05D14FF0010C0CFA00FCC2F8D3
:100B400010C0401C0828D1D31460B1F800C0BCF11B
:100B5000FF0F34DD546800202EE000F1080C4FF048
:100B6000010808FA0CF3B1F800C00CEA03069E4233
:100B700021D183004FF00F0C0CFA03F7BC4305FAA8
:100B800003FC4CEA040491F803C0BCF1280F05D122
:100B900000F1080C08FA0CF8C2F8148091F803C0B0
:100BA000BCF1480F07D100F1080C4FF0010808FA1A
:100BB0000CF8C2F81080401C0828CED35460BDE861
:100BC000F0814FF6FF710180022181700421C17014
:100BD00070470246002093680B4201D0012000E0DC
:100BE000002070470146886880B2704702460020A6
:100BF000D3680B4201D0012000E00020704701467D
:100C0000C86880B2704701617047416170470AB19E
:100C1000016100E041617047C16070474FF480326C
:100C20000A438261816182618269826970470246FA
:100C30000020424B18684FF68073184040EA0210BB
:100C400008433E4B186070473D49C8617047F0B596
:100C50000A46002300240021002500F00046B6F1DA
:100C6000004F02D1354EF16901E0344E7168C0F396
:100C7000034583B200F44016B6F5401F08D121F0B9
:100C800070612E4E766826F070662C4F7E6012E002
:100C900000F48016B6F5801F06D1032606FA05F487
:100CA000A14341F0706106E0460D360103FA06F6F5
:100CB000B14341F0706122B1460D360103FA06F6E8
:100CC000314300F00046B6F1004F02D11B4EF161F6
:100CD00001E01A4E7160F0BD30B500228B071C0F89
:100CE0000F2303FA04F2154B08338C1053F8243009
:100CF0009343124C08348D1044F8253023468C1051
:100D000053F824308C07240F00FA04F423430B4CCF
:100D100008348D1044F8253030BD0A49086070470A
:100D200000080140000C0140001001400014014087
:100D300000180140001C014000200140000001405B
:100D400000002042DC002042DD48006840F0010045
:100D5000DB49086008464068DA490840D8494860DD
:100D600008460068D8490840D54908600846006828
:100D700020F4802008600846406820F4FE004860A7
:100D80004FF41F0088607047CD49096821F4803115
:100D9000CB4A11601146096821F480211160B0F539
:100DA000803F03D0B0F5802F0ED106E0C44909681A
:100DB00041F48031C24A116007E0C149096841F439
:100DC000A021BF4A116000E000BF00BF704710B50E
:100DD00001460022002300204A11012A02D1B84C0A
:100DE000236806E0022A02D1B54C236A01E0B44C24
:100DF000636A01F01F02012494401C4201D00120CB
:100E000000E0002010BD38B500200090002400252F
:100E100000BF3120FFF7DBFF05460098401C009023
:100E20000098B0F5A06F01D0002DF2D03120FFF76F
:100E3000CEFF08B1012400E00024204638BD014661
:100E400000209F4A106820F0F80040EAC1001060BE
:100E500070479E490860704702460020984B5868CA
:100E600020F47C1042EA01031843954B5860704708
:100E700096490866704701460020914A506820F064
:100E800003000843506070478D48406800F00C0034
:100E90007047014600208A4A506820F0F00008435D
:100EA0005060704701460020854A506820F4E06099
:100EB00008435060704701460020814A506820F482
:100EC000605040EAC1005060704729B17C4A527AB4
:100ED00002437B4B5A7204E0794A527A8243784B40
:100EE0005A7270477A490860704701460020744A78
:100EF000506820F440400843506070470021754A14
:100F000011706F4A82F82010012802D0042808D1FD
:100F100003E001216F4A117004E005216D4A117050
:100F200000E000BF00BF70476B490860704764492C
:100F3000096A0143624A116270476749443908608F
:100F4000704730B500210022002400235C4D6D68FD
:100F500005F00C0121B1042905D0082923D105E0B1
:100F60005E4D056022E05E4D05601FE0544D6D68EA
:100F700005F47012524D6D6805F48034022505EBBE
:100F800092421CB9574D554305600BE04C4D6D68BE
:100F900015F4003F03D0544D5543056002E0504D19
:100FA0005543056002E04D4D056000BF00BF444D54
:100FB0006D6805F0F00109094C4D6B5C0568DD407A
:100FC00045603F4D6D6805F4E061090A474D6B5C73
:100FD0004568DD4085603A4D6D6805F46051C90A89
:100FE000424D6B5C4568DD40C560354D6D6805F46C
:100FF0004041890B3E4D6B5CC568B5FBF3F505615F
:1010000030BD29B12E4A526902432D4B5A6104E08A
:101010002B4A526982432A4B5A61704729B1284AA8
:1010200092690243264B9A6104E0254A9269824301
:10103000234B9A61704729B1214AD2690243204B60
:10104000DA6104E01E4AD26982431D4BDA617047BF
:1010500029B11B4AD2680243194BDA6004E0184AEE
:10106000D2688243164BDA60704729B1144A12697C
:101070000243134B1A6104E0114A12698243104B78
:101080001A61704714494039086070470F49C864B5
:1010900070470B49C87170470948406A40F080703A
:1010A00007494862704701460020054A92680A4293
:1010B00001D0012000E0002070470149887270478C
:1010C000001002400000FFF8FFFFF6FE0000424261
:1010D000D8004242201002408004424200127A00AE
:1010E000001BB70000093D00808D5B001800002048
:1010F0002800002010B50446BE48844208D10121D2
:101100008014FFF7A5FF0021A014FFF7A1FF16E050
:10111000B948844208D101210014FFF7A6FF00213D
:101120002014FFF7A2FF0AE0B448844207D101214E
:10113000C013FFF79AFF0021E013FFF796FF10BDE1
:1011400010B50022028802F441520B884C882343D8
:101150008C882343CC8823430C8923434C89234325
:101160008C892343CC8923431A430280838B4FF21B
:10117000FF74234083830B8A038210BD2DE9F04F57
:1011800085B005460C464FF0000902274FF00008D5
:101190004FF0010B0026B246A88B4FF240010840E9
:1011A000A88302202884B5F81C90A068022801D1E9
:1011B00000BF38E0A08810B94FF0010B01E04FF0FC
:1011C000020B8D48854200D100E000BF6846FFF762
:1011D000B8FEDDF800A0E088B0F5007F0AD14FEA44
:1011E0001A2000EB80004000A168B0FBF1F0401D28
:1011F00086B20BE04FEA4B10BAFBF0F000EB800038
:101200004000A168B0FBF1F0401D86B20A20B6FB99
:10121000F0F606F00108A6EB0800C0F34F074FF602
:10122000FF7000EA0828022F01DBFF2F02DD0227F2
:101230004FF00008E08840EA080038432884A0887E
:10124000A1890843618808432188084340F400606D
:1012500040EA0909A5F81C9005B0BDE8F08F00210F
:10126000018041808180C180018141818181C18172
:101270000721018270470021018041808180C18067
:101280000221816000218181704721B1028842F0F2
:101290004002028004E002884FF6BF731A400280C9
:1012A000704721B1828B42F48062828304E0828B9A
:1012B0004FF6FF331A408283704730B50024002375
:1012C0000C110125A540ABB21AB185881D4385805C
:1012D00002E085889D43858030BD1AB183880B4329
:1012E000838002E083888B438380704781817047CD
:1012F000014688897047A1F57E42FF3A04D00288F2
:1013000042F48072028004E002884FF6FF631A40C4
:101310000280704721B1828842F00402828004E09A
:1013200082884FF6FB731A408280704702884FF222
:10133000FF731A40028002880A43028070470188C6
:1013400041F480510180704721B1028842F400527B
:10135000028004E002884DF6FF731A400280704755
:1013600002460020012901D0108B00E0908A7047CE
:101370000146088A7047B1F5804F04D1028842F4D3
:101380008042028004E002884BF6FF731A4002801C
:1013900070470246002013890B4201D0012000E073
:1013A00000207047CA4302817047F0B50246002012
:1013B00000240023002501F00F070126BE40B4B22F
:1013C0000B1101269E40B3B2968806EA03051689E2
:1013D000264202D00DB1012000E00020F0BD10B582
:1013E000002201F00F040123A3409AB2D3430381EA
:1013F00010BD00000030014000380040003C0040BB
:1014000010B50446FB48844209D101218803FFF747
:101410001FFE00214FF48040FFF71AFE32E0F6482D
:10142000844209D101214804FFF71FFE00214FF437
:101430000030FFF71AFE25E0F048844209D101216F
:101440008804FFF712FE00214FF48020FFF70DFE05
:1014500018E0EB48844209D10121C804FFF705FEDA
:1014600000214FF40020FFF700FE0BE0E548844226
:1014700008D101210805FFF7F8FD00214FF4801085
:10148000FFF7F3FD10BD2DE9F04786B005460E4687
:101490000024A24600BFA1460027B08900B100BFCA
:1014A0002F462C8A4CF6FF700440F08804432C82AF
:1014B000AC894EF6F3100440B08831890843718935
:1014C00008430443AC81AC8A4FF6FF400440B08926
:1014D0000443AC8201A8FFF734FDC648874202D11D
:1014E000DDF810A001E0DDF80CA0A88910F4004F91
:1014F00008D00AEBCA0000EB0A1031684900B0FBC3
:10150000F1F807E00AEBCA0000EB0A103168890025
:10151000B0FBF1F86420B8FBF0F00401200964216D
:1015200001FB1089A88910F4004F08D0322000EB8D
:10153000C900B0FBF1F000F00700044308E03220DE
:1015400000EB09106421B0FBF1F000F00F00044340
:101550002C8106B0BDE8F0874FF4165101600021E0
:101560008180C18001810C214181002181817047EE
:1015700010B502460020108A4FF2FF0318400B8876
:101580004C8823438C882343CC8823431843108200
:1015900010BD0021018041808180C180704721B150
:1015A000828942F40052828104E082894DF6FF7301
:1015B0001A4082817047F0B50346002400260025BA
:1015C0000020A1F510676A3F00D100BF1846C1F3A3
:1015D000421401F01F06012707FA06F5012C01D17C
:1015E0000C3004E0022C01D1103000E014301AB1AC
:1015F00007682F43076002E00768AF430760F0BD4C
:101600001AB1838A0B43838202E0838A8B438382ED
:101610007047028A4FF6F0731A400282028A0A4328
:101620000282704782894FF2FF731A408281828959
:101630000A438281704721B1828942F0020282818D
:1016400004E082894FF6FD731A4082817047028A56
:101650004FF6DF731A400282028A0A430282704701
:1016600021B1028A42F48042028204E0028A4BF6EF
:10167000FF731A4002827047C1F3080282807047EC
:1016800001468888C0F308007047818941F0010154
:1016900081817047028BD2B20283028B42EA01221F
:1016A00002837047028B02F47F420283028B0A435B
:1016B0000283704721B1828A42F02002828204E0D4
:1016C000828A4FF6DF731A408282704721B1828A84
:1016D00042F01002828204E0828A4FF6EF731A40D1
:1016E0008282704721B1828A42F00802828204E03D
:1016F000828A4FF6F7731A408282704721B182893D
:1017000042F40042828103E08289C2F30E028281A8
:10171000704721B1828A42F40062828204E0828AA8
:101720004FF2FF731A4082827047828A4FF6FB7332
:101730001A408282828A0A438282704721B1828A59
:1017400042F00202828204E0828A4FF6FD731A4060
:101750008282704702460020B1F5007F00D100BFB1
:1017600013880B4201D0012000E00020704701F4F3
:101770000072B2F5007F00D100BFCA4302807047FB
:1017800070B502460024002300250020A1F5106654
:101790006A3E00D100BFC1F3421501F01F030126CC
:1017A00006FA03F3012D02D19689334006E0022D9B
:1017B00002D1168A334001E0968A33400C1201268A
:1017C00006FA04F41688344013B10CB1012000E08D
:1017D000002070BD10B500220023A1F510646A3C02
:1017E00000D100BF0A1201249440A3B2DC4304805C
:1017F00010BD000000380140004400400048004097
:10180000004C00400050004001684FF6FE7211404D
:1018100001600021016041608160C1608C498842A3
:1018200008D18B490839496841F00F01884A083AC4
:1018300051608AE086491431884208D184490839C8
:10184000496841F0F001824A083A51607DE08049E0
:101850002831884208D17E490839496841F47061CD
:101860007B4A083A516070E079493C31884208D19E
:1018700077490839496841F47041754A083A51601E
:1018800063E073495031884208D171490839496889
:1018900041F470216E4A083A516056E06C49643157
:1018A000884208D16A490839496841F47001684A98
:1018B000083A516049E066497831884208D1644964
:1018C0000839496841F07061614A083A51603CE06A
:1018D0006049884206D1011F096841F00F01021FCB
:1018E000116032E05B491431884208D15949091F1F
:1018F000096841F0F001574A121F116025E055496F
:101900002831884208D15349091F096841F47061A0
:10191000504A121F116018E04E493C31884208D1EC
:101920004C49091F096841F470414A4A121F11606D
:101930000BE048495031884207D14649091F0968E0
:1019400041F47021434A121F1160704710B5002204
:10195000026847F6F0739A430C6A8B6823430C695C
:1019600023434C6923438C692343CC6923434C6A4A
:1019700023438C6A23431A430260CB6843600B689D
:1019800083604B68C36010BD0021016041608160CD
:10199000C160016141618161C16101624162816235
:1019A000704721B1026842F00102026004E002685F
:1019B0004FF6FE731A40026070471AB103680B437A
:1019C000036002E003688B43036070474160704727
:1019D0000146486880B2704701460020002211F09D
:1019E000805F03D01B4B083B1A6802E0184B083B92
:1019F0001A680A4201D0012000E00020704710F070
:101A0000805F03D01349091F086002E010490839BC
:101A10004860704701460020002211F0805F03D02B
:101A20000C4B083B1A6802E0094B083B1A680A4253
:101A300001D0012000E00020704710F0805F03D04B
:101A40000449091F086002E00149083948607047ED
:101A5000080002400804024001460020FE4A1068C7
:101A600000F03800084310607047FB49096821F016
:101A70000801F94A11601146096801431160704775
:101A8000F549096821F01001F34A1160114609680F
:101A9000014311607047F148EF494860F0484860E1
:101AA0007047EE48EC494860ED4848607047EA48A6
:101AB000006940F08000E84908617047E648006925
:101AC00040F08000E449086170470420E249C96899
:101AD00011F0010F01D001200EE0DF49C96811F0BB
:101AE000040F01D0022007E0DB49C96811F0100F94
:101AF00001D0032000E00420704700B50246042313
:101B0000FFF7E3FF034603E0FFF7DFFF0346521E44
:101B1000012B01D1002AF7D102B90523184600BDD7
:101B200030B5044604254FF43020FFF7E6FF0546A4
:101B3000042D17D1C848006940F00200C649086169
:101B400008464461006940F0400008614FF43020CD
:101B5000FFF7D3FF0546C048006941F6FD71084014
:101B6000BD490861284630BD10B504244FF430202B
:101B7000FFF7C3FF0446042C16D1B748006940F0B4
:101B80000400B54908610846006940F0400008615A
:101B90004FF43020FFF7B1FF0446AF48006941F62B
:101BA000FB710840AC490861204610BD00B50246F3
:101BB0000423FFF78AFF034603E0FFF786FF03468F
:101BC000521E012B01D1002AF7D102B90523184674
:101BD00000BD10B504244FF43020FFF7E7FF0446A2
:101BE000042C16D19C48006940F004009A49086111
:101BF0000846006940F0400008614FF43020FFF7CC
:101C0000D5FF04469448006941F6FB7108409249AB
:101C10000861204610BD00208F49C96911F0020FEC
:101C200001D0012000E00020704730B5A525042434
:101C3000FFF7F1FF00B100254FF43020FFF75DFF03
:101C40000446042C3AD185488349886084488860DA
:101C50000846006940F0200008610846006940F02D
:101C6000400008614FF43020FFF747FF0446042C82
:101C70001BD17948006941F6DF7108407649086157
:101C80000846006940F01000086176480580E002CF
:101C9000FFF733FF0446052C10D06F48006941F66A
:101CA000EF7108406C49086108E0052C06D06A48CD
:101CB000006941F6EF71084067490861204630BD70
:101CC00078B506460C46042500200090E802FFF790
:101CD00014FF0546042D24D15F48006940F001003F
:101CE0005D4908613480E802FFF707FF0546042DCF
:101CF00010D1B01C0090200C00990880E802FFF77A
:101D0000FCFE05465448006941F6FE710840524900
:101D1000086106E05048006941F6FE7108404E49EE
:101D20000861284678BD70B504460D460426F002C9
:101D3000FFF7E3FE0646042E11D14748006940F044
:101D40000100454908612580F002FFF7D6FE0646EE
:101D50004148006941F6FE7108403F49086130463C
:101D600070BD70B505460E460424E002FFF7C5FEBF
:101D70000446042C17D139483749886038488860B0
:101D80000846006940F0100008612E80E002FFF76D
:101D9000B4FE0446052C06D02F48006941F6EF71C9
:101DA00008402D490861204670BD2DE9F0430446E6
:101DB0004FF6FF763746B046B1460425E443E6B217
:101DC000C4F30727C4F307484FEA1469E802FFF792
:101DD00094FE0546042D49D120481F4988602048BB
:101DE00088600846006940F010000861FF2E06D0A8
:101DF0001C4808300680E802FFF77FFE0546042DE8
:101E000008D1FF2F06D017480A300780E802FFF7F5
:101E100074FE0546042D0AD1B8F1FF0F07D0114812
:101E20000C30A0F80080E802FFF767FE0546042D9D
:101E30000AD1B9F1FF0F07D00A480E30A0F8009080
:101E4000E802FFF75AFE0546052D0FD0024800694B
:101E500041F6EF71084007E000200240230167458A
:101E6000AB89EFCD00F8FF1F664908612846BDE841
:101E7000F08330B5054604244FF43020FFF73DFED3
:101E80000446042C41D160485E4988605F48886000
:101E90000846006940F0200008610846006940F0EB
:101EA000400008614FF43020FFF727FE0446042C61
:101EB00022D15448006941F6DF7108405149086158
:101EC0000846006940F0100008611DB1002050492B
:101ED000088002E0A5204E4908804FF43020FFF72B
:101EE0000CFE0446052C10D04648006941F6EF71FF
:101EF00008404449086108E0052C06D041480069C3
:101F000041F6DF7108403F490861204630BDF0B519
:101F100005460E46174604243B483A4988603B482C
:101F20008860E002FFF7E9FD0446042C19D135482A
:101F3000006940F010003349086147F0F800304371
:101F400028433349891C0880E002FFF7D6FD044688
:101F5000052C06D02B48006941F6EF71084029494D
:101F600008612046F0BD2748C069800870472548B1
:101F7000006A704700202349096811F0200F01D042
:101F8000012000E00020704729B11E4A1269024377
:101F90001C4B1A6104E01B4A12698243194B1A61F7
:101FA000704701460020012908D1164AD26912F073
:101FB000010F01D0012008E0002006E0114AD2689C
:101FC0000A4201D0012000E0002070470D49C8609E
:101FD000704704200B49C96811F0010F01D001209E
:101FE0000EE00849C96811F0040F01D0022007E093
:101FF0000449C96811F0100F01D0032000E004204B
:10200000704700000020024023016745AB89EFCDF7
:1020100000F8FF1F0E49086070470D49486070477F
:102020000B49886070474AF6AA2009490860704742
:102030004CF6CC4006490860704701460020044A2F
:10204000D2680A4201D0012000E000207047000061
:102050000030004008B54FF48070ADF8000010204B
:102060008DF8030003208DF802006946FE48FEF754
:102070001FFD0020FD49086008BD08B54FF48060D1
:10208000ADF8000010208DF8030003208DF8020049
:102090006946F748FEF70CFD4FF40060ADF800000C
:1020A00010208DF8030003208DF802006946F048E7
:1020B000FEF7FEFC4FF48050ADF8000010208DF8C4
:1020C000030003208DF802006946E948FEF7F0FCA2
:1020D00008BD08B54020ADF8000010208DF80300C1
:1020E00003208DF802006946E248FEF7E1FC4FF458
:1020F0000040ADF8000010208DF8030003208DF89B
:1021000002006946DA48FEF7D3FC08BD08B538205E
:10211000ADF8000018208DF8030003208DF80200B0
:102120006946D548FEF7C4FC8020ADF800001020B9
:102130008DF8030003208DF802006946CE48FEF7B3
:10214000B7FC8021CC48FEF75EFD8020ADF8000092
:1021500010208DF8030003208DF802006946C44862
:10216000FEF7A6FC8021C248FEF74DFD08BD08B56C
:102170000820ADF8000010208DF8030003208DF832
:1021800002006946BD48FEF793FC0020BC49086088
:1021900008BD08B50820ADF8000000208DF8030048
:1021A00003208DF802006946B448FEF781FC08BDA3
:1021B00008B50120ADF8000010208DF803000320C1
:1021C0008DF802006946AD48FEF772FC0220ADF8BA
:1021D000000010208DF8030003208DF802006946EE
:1021E000A648FEF765FC4FF48070ADF800001020A3
:1021F0008DF8030003208DF8020069469E48FEF723
:1022000057FC4FF40070ADF8000010208DF803006B
:1022100003208DF8020069469748FEF749FC01212A
:102220009648FEF7F0FC08BD08B50120ADF80000A7
:1022300028208DF8030003208DF8020069468F489E
:10224000FEF736FC0220ADF8000028208DF80300D0
:1022500003208DF8020069468848FEF729FC4FF4F8
:102260008070ADF8000028208DF8030003208DF861
:10227000020069468048FEF71BFC4FF40070ADF881
:10228000000028208DF8030003208DF80200694625
:102290007948FEF70DFC08BD08B501210420FEF7C2
:1022A000BDFEFF20ADF8000010208DF803000320D4
:1022B0008DF8020069466C48FEF7FAFB0121082000
:1022C000FEF7ACFE4FF44050ADF8000028208DF82A
:1022D000030003208DF8020069466748FEF7E8FB1B
:1022E0004FF44040ADF8000010208DF803000320AB
:1022F0008DF8020069466048FEF7DAFB01214020B4
:10230000FEF78CFE4020ADF8000010208DF8030091
:1023100003208DF8020069465848FEF7C9FB0020EB
:10232000584908605849C1F8B801584908605849E7
:10233000086001F10401086001F10401086001F185
:102340000401086001F10401086001F10401086062
:1023500001F10401086001F10401086008BD08B53D
:1023600001210420FEF75AFEFF20ADF800000020F6
:102370008DF8030003208DF8020069463A48FEF705
:1023800097FB01210820FEF749FE4FF44050ADF8BD
:10239000000000208DF8030003208DF8020069463C
:1023A0003548FEF785FB4FF44040ADF800000020B3
:1023B0008DF8030003208DF8020069462E48FEF7D1
:1023C00077FB01214020FEF729FE4020ADF80000F8
:1023D00000208DF8030003208DF80200694627488D
:1023E000FEF766FB08BD08B50220ADF8000000202E
:1023F0008DF8030069461F48FEF75AFB0120ADF82F
:10240000000000208DF8030069461A48FEF750FBD3
:1024100008BD08B50220ADF8000000208DF80300CB
:1024200069461448FEF744FB08BD08B50120ADF825
:10243000000000208DF8030069460E48FEF738FBC7
:1024400008BD08B58020ADF8000028208DF80300F5
:1024500069460848FEF72CFB4FF48070ADF8000089
:102460006946044816E0000000080140A00121422E
:102470000014014000100140000C01400018014010
:102480008C0123429801234200802142BC812142D9
:1024900080012142FEF70CFB4FF40070ADF8000004
:1024A0006946FE48FEF704FB08BD08B50220ADF8FA
:1024B000000010208DF8030003208DF8020069460B
:1024C000F748FEF7F5FA0020F649086008BD08B5A0
:1024D0004FF40070ADF8000018208DF80300694635
:1024E000F148FEF7E5FA4FF48060ADF800000420F3
:1024F0008DF803006946EC48FEF7DAFA08BD08B526
:102500004FF40070ADF8000000208DF8030069461C
:10251000E548FEF7CDFA4FF48060ADF800000020EA
:102520008DF803006946E048FEF7C2FA4FF4807068
:10253000ADF8000000208DF8030003208DF80200A4
:102540006946D948FEF7B4FA08BD08B54FF4005003
:10255000ADF8000010208DF8030003208DF8020074
:102560006946D248FEF7A4FA4FF48040ADF8000067
:1025700010208DF8030003208DF802006946CB4837
:10258000FEF796FA4FF40060ADF8000028208DF8B1
:1025900003006946C548FEF78BFA4FF40051C34863
:1025A000FEF731FB4FF48041C048FEF72CFB08BD1D
:1025B00008B54FF40050ADF8000018208DF8030066
:1025C00003208DF802006946B548FEF771FA08BD90
:1025D00008B54FF40040ADF8000010208DF803005E
:1025E00003208DF802006946AD48FEF761FA4FF40A
:1025F0000041AB48FEF709FB08BD08B54FF4005099
:10260000ADF8000000208DF8030003208DF80200D3
:102610006946A348FEF74CFA08BD08B54FF40040E0
:10262000ADF8000010208DF8030003208DF80200A3
:1026300069469D48FEF73CFA00209D49086008BDA8
:1026400008B58020ADF8000010208DF803000320AD
:102650008DF8020069469548FEF72AFA0020954950
:10266000086008BD08B58020ADF8000010208DF886
:10267000030003208DF8020069468C48FEF718FA23
:1026800000208C49086008BD08B50220ADF80000A4
:1026900010208DF8030003208DF802006946804861
:1026A000FEF706FA00207F49086008BD08B54FF420
:1026B0008060ADF8000018208DF8030003208DF82D
:1026C000020069467C48FEF7F3F94FF40060ADF86C
:1026D000000004208DF8030003208DF802006946F5
:1026E0007548FEF7E5F94FF48070ADF80000102052
:1026F0008DF8030003208DF8020069466B48FEF751
:10270000D7F901206D49086008BD08B58020ADF8F3
:10271000000000208DF8030003208DF802006946B8
:102720006248FEF7C5F94FF48060ADF80000002064
:102730008DF8030003208DF8020069465E48FEF71D
:10274000B7F94FF40060ADF8000000208DF80300E9
:1027500069465948FEF7ACF94FF48070ADF80000B7
:1027600000208DF8030003208DF8020069464F48D1
:10277000FEF79EF901205149086008BD08B5012007
:10278000ADF8000010208DF8030003208DF8020042
:1027900069464948FEF78CF94FF40060ADF8000037
:1027A00010208DF8030003208DF8020069463F4891
:1027B000FEF77EF90020424908604249C1F88001D5
:1027C00008BD08B54FF40060ADF8000010208DF88A
:1027D000030003208DF8020069463348FEF768F9CC
:1027E00000203949086008BD10B54FF400612E483B
:1027F000FEF7FCF908B9012000E00020044622465B
:102800004FF400612848FEF702FA10BD08B52020F9
:10281000ADF8000010208DF8030003208DF80200B1
:1028200069461E48FEF744F900202849086008BDA3
:1028300008B54FF40060ADF8000010208DF80300DB
:1028400003208DF8020069461848FEF731F9002090
:102850001B49086008BD08B54FF40060ADF80000E2
:1028600004208DF8030003208DF8020069460E480D
:10287000FEF71EF908BD704708B54FF2FF70ADF8BE
:10288000000000208DF8030069460748FEF710F9A4
:102890004FF6FF70ADF80000002019E00010014075
:1028A00000140140848122420008014000180140C8
:1028B000BC0121429C012342000C0140A0012342A3
:1028C000AC01234200802142AC012142940122420A
:1028D0008DF8030069461748FEF7EAF84FF6F770DF
:1028E000ADF8000000208DF8030069461248FEF79D
:1028F000DFF80820ADF8000004208DF803006946D9
:102900000D48FEF7D5F84FF6FF70ADF80000002037
:102910008DF8030069460948FEF7CAF847F6F770D4
:10292000ADF8000000208DF8030069460448FEF76A
:10293000BFF808BD000C0140001001400014014028
:102940000018014070B504460D46002305E02678C6
:102950002E706D1C641C5E1CF3B29342F7DB70BDDD
:102960000146088870472DE9F04105460E46174696
:10297000002407E036F814102846FFF7D4F9AD1C00
:10298000601C84B2BC42F5DBBDE8F08130B5034683
:102990000C461546002207E01846FFF7E1FF24F831
:1029A00012009B1C501C82B2AA42F5DB30BD2DE9FF
:1029B000F04106460F461446204604EBD0714910FC
:1029C000A4EB4101012905D104EBD0714910491C48
:1029D0008DB203E0204604EBD0714D10FFF75BF899
:1029E0002A4631463846FFF7BEFFFFF760F8BDE8DC
:1029F000F08110B5D648006800285FD0D54800782F
:102A000000285CDD00BFD3480078401DD04909682C
:102A10008842F8D8CF48C078C8B9FFF7E5FE00244F
:102A20000DE0201DCB49085CCB49CC4A1268885484
:102A3000CA480068401CC9490860601CC4B2C54847
:102A40000078A042EDDC0020C149086013E0C148D5
:102A5000C07805280FD1BF480079C1490870BD482A
:102A600040794870BB4880798870BA48C079C8708E
:102A70000020B7490860B9480068B0F5006F13D16D
:102A8000FFF7B2FE4FF40062B6480168B248FFF7A4
:102A90008EFFB448006800F50060B249086000206D
:102AA000AE490860FFF7A0FEAA490978091DA94AA6
:102AB00088180121FDF706FDFFF796FE31E0A448D6
:102AC000006805282DD1A348407850BBA1488078E4
:102AD00038BBA048C078012823D19E480079FF2840
:102AE0001FD1FFF781FE9D48008882B29D48016892
:102AF0009948FFF75CFFFFF777FE9A48006897490F
:102B0000096808449749086000209449086001203A
:102B10009549087001218F48001DFDF7D3FCFFF790
:102B200063FEFFF761FE10BD10B5FFF75DFE88483C
:102B30000068002843D0874800788C49097888428B
:102B40003AD18348006807282ED1824840788749C7
:102B50004978884224D17F4880788449897888429E
:102B60001ED17C48C0788149C978884218D17948FB
:102B700000797E490979884212D1764840797B49AB
:102B8000497988420CD1734880797849897988429B
:102B900006D100206E490860FFF726FE012010BD17
:102BA00000206B4908600AE069480068072806D9D8
:102BB00000206749086002E00020654908600020A5
:102BC000EDE710B56A4CFEF766FFFFF70DFE00BF9C
:102BD00006E0FFF709FE2046FEF7A2FF04F50064B9
:102BE00064488442F5D3FFF7FFFDFEF760FF10BD98
:102BF00070B505460024FEF74EFFFFF7F5FD5E4871
:102C0000FEF78EFFFFF7F0FD10225C495A48FFF7F0
:102C1000AAFEFFF7E9FDFEF74AFF70BD10B50446B6
:102C2000206857490840B0F1005F08D160685549F5
:102C300008602068FDF78FFA52480068804710BD91
:102C400000BFFFF7D1FDFFF7BCFF0020404908603F
:102C500042490860464843490860002042490870DC
:102C600007214948FDF72EFC16E003E0FFF7BCFD05
:102C7000FFF7BFFE3C4800780028F7D008E0FFF7D8
:102C8000B3FD38480068FFF7B3FF3948FFF7C6FFC8
:102C9000354800780128F2D0E7E710B572B6002178
:102CA0003A48FEF77CFC0520FDF7E2FA002038499F
:102CB00008604FF00A00FDF7DBFA002080F310886F
:102CC00000BF2B48FFF7AAFF10BD10B5FFF78CFD22
:102CD000FEF7E1FE10222F492748FFF757FEFEF7C7
:102CE000E6FEFFF781FD00240AE02A4830F81400D0
:102CF000224931F81410884200D003E0601CC4B2AD
:102D0000102CF2DB00BF0F2C03DDFFF76DFD01205F
:102D100010BDFFF769FD0020FAE710B540F225511C
:102D20001A48FEF72DFD88B11848FEF7A9FC09499D
:102D3000074A1268885406480068401C0449086025
:102D400008460068642801D30020086010BD000018
:102D50003800002072010020420200203C000020C8
:102D6000300000202C00002034000020B42F000888
:102D7000008000080000080800780008BC2F000848
:102D80000000FE2F40000020A62F00080048004051
:102D900084812242A60A002010B501217C20FEF782
:102DA0003DF901210846FEF739F9FFF70AFD4FF416
:102DB00000616248FDF71AFF08B9012000E0002019
:102DC000044622464FF400615C48FDF720FFFFF700
:102DD0009DF9FFF76AFBFFF7CAF90120584908601F
:102DE000FFF7E6F9FFF7CAFCFFF7AFFBFFF7E0FBE1
:102DF000FFF7EEFBFFF725FBFFF70FFCFFF7AFFA3E
:102E0000FFF71EFCFFF737FD10BD08B5012150206C
:102E1000FEF704F903208DF8020048208DF8030026
:102E20000120ADF8000069464648FDF741FE4FF429
:102E30000070ADF8000069464348FDF739FE1020E8
:102E40008DF803000220ADF8000069463D48FDF70B
:102E50002FFE4FF48060ADF8000069463A48FDF758
:102E600027FE4FF480613848FDF7CDFE022135483A
:102E7000FDF7C9FE01203549086008BD10B50121E4
:102E80007C20FEF7CBF801210846FEF7C7F8FFF7D4
:102E90006EF901202A490860FFF78AF9FFF76EFCF6
:102EA000FFF753FBFFF7CDFAFFF7E5FC10BD10B5B8
:102EB0004FF48030FDF768FFFDF7A5FF0446012CB5
:102EC00010D10020FDF7E5FFA002FDF7EBFF002089
:102ED000FDF7F1FF0120FDF7CEFF00BFFDF7D4FFA6
:102EE0000428FBD110BD10B545F25550FFF792F8FC
:102EF0000520FFF792F84FF42F70FFF791F8FFF7D6
:102F000092F8FFF795F810BD10B5FFF78CF810BDDB
:102F100010B50121C803FEF78EF801210846FEF71F
:102F20007DF801210A48FDF792FEFDF731FB10BD47
:102F300010B54FF4E130FDF7C7F910BD00080140AE
:102F40008C012342001001400018014094012242EC
:102F500000023000421C10F8011B0029FBD1801A2E
:102F600070470000064C074D06E0E06840F00103A2
:102F700094E8070098471034AC42F6D3FDF7DCF82C
:102F8000DC2F0008FC2F000802E008C8121F08C14F
:102F9000002AFAD170477047002001E001C1121FDA
:102FA000002AFBD170470301AA55038D3E0301059A
:102FB0000A035C37040255AA03C9FA000000110095
:102FC0002200330044005500660077008800990015
:102FD000AA00BB00CC00DD00EE00FF00FC2F0008C3
:102FE0000000002044000000882F00084030000846
:102FF000440000208C120000982F00080000000000
:10300000001BB700000000000000000001020304E4
:10301000060708090000000001020304010203047E
:10302000060708090204060800000000000000006E
:103030000000000000000000000000000000000090
:0400000508000131BD
:00000001FF
